:1078000011241FBECFEFDAE0DEBFCDBFF2C04101D1
:1078100042144505560455026403740300001E9586
:1078200087020110030000C18081C106C0FF0A0069
:107830000CA10185037508150026FF00954009017C
:107840008102954009029102C004030904380341F2
:107850000072006400750069006E006F0020004D2A
:10786000006900630072006F00200062006F006F0B
:107870000074006C006F00610064006500720020FD
:1078800000200020001803410072006400750069A8
:10789000006E006F0020004C004C004300120100FD
:1078A00002020000404123350000010102000112E4
:1078B00001000200000040412335000001010200E8
:1078C00001090264000301008032080B0002020279
:1078D000010009040000010202000005240010015B
:1078E0000524010101042402020524060001070504
:1078F000810310004009040100020A00000007058E
:107900000202400000070583024000000904020053
:107910000103000000092101010001221E000705EA
:1079200084034000400020918A0130918B012C5F3C
:107930003F4F30938B0120938A01C901892F9927EA
:107940008695982F803418F08FE7891B982F990F10
:10795000921710F447980895479A0895769A289AAE
:1079600081E08093E0001092E200EE27FF27099467
:1079700008950F931F93CF93DF93982FEB01042F5C
:1079800010E088E76030780730F411E083E0FB0115
:1079900080935700E895892F68E071E0402FF8D078
:1079A000112311F107B600FCFDCF402F4695FE01D3
:1079B000A8E0B1E020E031E009C08D919D910C017B
:1079C00030935700E895112432962F5F2417A8F3BF
:1079D00085E0FE0180935700E89507B600FCFDCFD7
:1079E00081E180935700E895DF91CF911F910F912E
:1079F000089588E10FB6F8948093600010926000BB
:107A00000FBE769A289A47983F9A209A6E9A90E8E5
:107A1000909361001092610081E885BF95BF9FD06F
:107A200084E18093880180E180938901E0E0F0E0C7
:107A3000859194918F5F9F4F19F081E080938F0122
:107A4000EE24FF24BB24B39454EFC52E51E0D52E71
:107A50000ED2082F8EE098E7FC0124913196029611
:107A60004491201711F02223B9F71092910110923E
:107A7000900182E068E071E08BD0013479F460918C
:107A800008016058633028F0683111F064E001C0EB
:107A900063E0C62FD0E0CF5DD7480EC0063571F445
:107AA00080910801803311F011E022C080910A0119
:107AB000C82FD0E0C25ED74811E022C0053721F4BC
:107AC00013E0CEE1D8E71CC0053539F4E090080199
:107AD000F0900901EE0CFF1C0AC0043631F482E07C
:107AE000B7014091090145DF02C0043721F010E0E1
:107AF000C5E2D8E705C010910901E701E10EF11CCC
:107B0000B6D18097B1F483E068E871E041E050E0DD
:107B100059D0112329F0412F50E083E8BE0152D003
:107B200083E469E871E041E050E04CD0013509F0B0
:107B30008FCFD0929101C0929001B0928F01EE242C
:107B4000FF2486CFFC01289884E680938D0104C031
:107B50008091F100819361506623D1F708951092CE
:107B600091011092900110928E0110928F0181E08C
:107B70008093D70080EA8093D80082E189BD09B460
:107B800000FEFDCF80E98093D8001092E0000895B8
:107B9000FB018093E90024E69BE611C08091E80098
:107BA00085FFFCCF289820938D018091F10081936F
:107BB0008091E80085FD02C09093E8004150442385
:107BC00069F70895982FFB01282F20728770809302
:107BD000E90064E63AE317C08091E80085FFFCCF36
:107BE00097FF02C0849101C080813196211180E00D
:107BF000769860938C018093F1008091E80085FD78
:107C000002C03093E800415050408FEF4F3F58077B
:107C100019F796FF03C08AE38093E80008958091E6
:107C20009301813299F4769884E680938C0120E068
:107C300030E003C080818093F100F901E050FF4FF4
:107C40002F5F3F4F28303105A9F714C0803261F40F
:107C50008091E80082FFFCCF80E091E067E072DF76
:107C60008BEF8093E80006C0823221F4809194016A
:107C70008093070181E0089520919501223261F1FE
:107C8000213081F48091980190919901089711F425
:107C900020939A0180919A01882309F04AC0EFEA63
:107CA000F8E749C0223021F484E6E1ECF8E717C098
:107CB000233009F03CC080919401882319F4E9E451
:107CC000F8E739C0823019F4EDE4F8E734C08130C8
:107CD00071F5E5E8F8E72FC081E0EBE2F8E7909175
:107CE0009801382F981708F4392F90918C0120E0D3
:107CF0004EEF8091E8008570E1F38091E80082FD0D
:107D000012C02F5F849176988093F100822F8F7339
:107D100011F44093E800319694E6231750F39093C2
:107D20008C0181E0089590938C0180E0089580E0BB
:107D30000895EDE9F8E78491D2CF1092E90080919F
:107D4000E80083FF61C082E991E068E0FBDE82EF3A
:107D50008093E8008091920187FF05C08091E80040
:107D600080FFFCCF03C08EEF8093E80080919301E9
:107D7000853051F48091E80080FFFCCF8091940120
:107D800080688093E30039C08930E1F480919401E8
:107D900080938E01E7E2F8E791E031E026E39093EB
:107DA000E9003093EB0084918093EC002093ED0088
:107DB0009F5F3196953099F78EE78093EA00109295
:107DC000EA001BC0883049F490918E01769884E6D1
:107DD00080938C019093F10010C0882339F4769839
:107DE00084E680938C011092F10007C0863011F474
:107DF00043DF01C014DF882321F08EEF8093E80079
:107E0000089581E28093EB0008958091E100109243
:107E1000E100282F83FF0CC01092E90081E08093DD
:107E2000EB001092EC0082E38093ED0010928E0143
:107E300022FF1CC080918C01882331F081508093F7
:107E40008C01882309F4769A80918D01882331F082
:107E5000815080938D01882309F4289A80918F01A5
:107E6000882321F4109291011092900108951F939C
:107E7000CF93DF9312E0C0E9D1E05FDFC6DF10935C
:107E8000E9008091E80085FF13C0289884E680937C
:107E90008D019091F1008091E80085FD03C08BE693
:107EA0008093E800892F90E0DF91CF911F91089592
:107EB000809190019091910101979093910180930D
:107EC00090018091900190919101892B09F446DDF8
:0A7ED000CE010197F1F727DDD0CFB6
:087EDA0000E1000000000000BF
:040000030000780081
:00000001FF
